:1000000000308A00F82800000A108A100A118207BE
:1000100044346F346234613420346D3465347A345E
:100020006934203473347434693473346B346E340B
:100030007534743469346D342034623479346C34FA
:1000400061342034253435342E343334773420343D
:1000500073342E340A340D34003424308400831376
:100060000008031944280130F800BF30F70064008D
:10007000F70B3728F80B35284A30F700F70B3E28E6
:1000800000006400800B33285929F701F801F901B9
:10009000FA01BC01BD01BE01BF013B083A043904AD
:1000A0003804031983282030C0000310B40DB50DA7
:1000B000B60DB70DBC0DBD0DBE0DBF0D3B083F020B
:1000C000031D6C283A083E02031D6C2839083D02C6
:1000D000031D6C2838083C02031C7D283808BC022C
:1000E0003908031C390FBD023A08031C3A0FBE023F
:1000F0003B08031C3B0FBF020314F70DF80DF90D6D
:10010000FA0DC00B55283C308400831300340408DA
:10011000AC003B30B3009A30B200CA30B100B0013D
:100120000A30AE002B08031DAC032A08B7002908CB
:10013000B6002808B5002708B4003308BB00320811
:10014000BA003108B9003008B80045200008A700FF
:10015000840A0008A800840A0008A900840A00088C
:10016000AA00FD308407F708031DC9282B0A2E02B8
:100170000319C9282C080319CA280F392E0203199C
:10018000C3280318DF28AC1BDF282C1BCA2820300B
:10019000DA28AC012B082E02031DD9287708AC0001
:1001A0002E300C1ED12899002C08F7002030AC0509
:1001B00000303030F70777080C1EDC289900330830
:1001C000B7003208B6003108B5003008B400BB01F2
:1001D000BA01B9010A30B80045207A08B30079089D
:1001E000B2007808B1007708B000AE0B95288F29CF
:1001F000840183131F308305193083169900A630BC
:10020000980090308312980083161F149F141F15B6
:100210009F1107309C00FF308312A00083161F142B
:100220009F141F159F1183121F108316091283122A
:100230009412A0122008831687008312201620082B
:10024000831687008312A0112008831687000130CF
:10025000831294000030831694000108C7390838CF
:100260008100831290010030F80092000030831664
:10027000920006309C0005080338850064000230B7
:10028000F700F70B412944291C0883120D13A030F5
:1002900083169D008312A310231483161C1B4E2962
:1002A0008312A2010130A100231C6E290130A40099
:1002B0002D2883161C1F5F298312A3148316003078
:1002C0001C1F01308312A4000030A3180130240544
:1002D000031D2310A10A0319A20A54290130210287
:1002E000A4002208A5000030031C0130A502A601CD
:1002F00026080420A60AF70077080C1E7D2999001D
:100300001A302602031D782905308400AA01A901AC
:100310002508A8002408A7000330AB0087281F3059
:10032000A70027080420A70AF70077080C1E9629C3
:0E033000990024302702031D91294B296300F8
:02400E00393F38
:00000001FF
